:100000000128831605108510061286120613861421
:100010000615861583120510851096019701980123
:1000200099019A019B019C019D019E019F01FF2066
:1000300006192A289D0AF4308C0001308D006821B1
:100040001D08043C00300319FF3EFF3903192A281C
:100050009D0186121D08013C00300319FF3EFF3947
:10006000031935280616061386121D08023C0030B7
:100070000319FF3EFF39031940280617061286129E
:100080001D08033C00300319FF3EFF3903194B28BC
:10009000861606130612861865280514C8308C00CB
:1000A00000308D0068210321F4308C0001308D0078
:1000B00068211121C8308C0000308D0068210510A6
:1000C000D0308C0007308D0068218619E428051493
:1000D0009F0AF4308C0001308D0068211F08143C09
:1000E00000300319FF3EFF39031978289F010321CF
:1000F0001E08003C00300319FF3EFF390319832816
:1001000001309E0003211D08013C00300319FF3E11
:10011000FF3903199328F4308C0001308D006821D9
:100120001F219D0106121D08023C00300319FF3EED
:10013000FF390319A928F4308C0001308D006821A3
:100140001F21F4308C0001308D0068211F219D019A
:1001500006131D08033C00300319FF3EFF39031945
:10016000C728F4308C0001308D0068211F21F43045
:100170008C0001308D0068211F21F4308C0001308B
:100180008D0068211F219D01861201309C001C08F2
:10019000003C0301031CFF3E0319E4289C0A861659
:1001A00064308C0000308D006821861264308C0031
:1001B00000308D0068211C08393C00300319FF3ED7
:1001C000FF390319E4289C01861DFD289F019C012D
:1001D0001E08013C00300319FF3EFF390319FC28BB
:1001E0009E01F4308C0001308D0068211121C8304F
:1001F0008C0000308D006821051018280128061297
:100200008612061308009601970148309A00F430D0
:100210008C0001308D000C0898000D0899002D21EC
:100220000800960197012B309A00D1308C000330E2
:100230008D000C0898000D0899002D2108009601EA
:10024000970139309A0003308C0003308D000C0880
:1002500098000D0899002D21080016088C00170839
:100260008D0018088E0019088F00572103194029A6
:10027000960A0319970A9B0141219B014C212D29C4
:1002800008001B081A0203010318FF3E03194B293B
:100290009B0A8514412908001B081A020301031850
:1002A000FF3E031956299B0A85104C2908000D08AA
:1002B0000F02031D5F290C080E020319642903189D
:1002C00064298C018D010800FF388C008D00080026
:1002D0008E018F01133090001F309100910B6E2919
:1002E000900B6C2928309000900B74298E0A03190A
:1002F0008F0A0C080E02031D6A290D080F02031D48
:040300006A2908005E
:00000001FF
